:100000000C9430050C9477050C9477050C947705C7
:100010000C9477050C9477050C9477050C94770570
:100020000C9477050C9477050C94930C0C94650D47
:100030000C94621C0C9477050C9477050C9477054E
:100040000C9477050C9477050C9477050C94770540
:100050000C9477050C94021D0C9477050C9477058D
:100060000C9477050C9477050C9477050C94770520
:100070000C9477050C9477050C9477050C94770510
:100080000C9477050C9477050C9477050C94770500
:100090000C9477050C9477050C9477050C947705F0
:1000A0000C9477050C9477050C947705D20DF40D1C
:1000B000E20EF40DE20E390E5C0EE20EB10EC40E2D
:1000C000EA11EA11191219127712B512CF14CF14CE
:1000D000CE12CF14CF13CF13A314CF14CF14BA144E
:1000E0008080352B787939808080210877060780D9
:1000F0008080201A7A1B168080801E802980808054
:100100008080808080808080808022158019098096
:1001100080801F147B1D0480808023172C050A809B
:100120008080260C00360E808080251876100D8089
:100130008080241C80110B80808027127E370F80E6
:1001400080802A804F7D2880808074305152328098
:1001500080802D137C38338080802E2F5075348022
:100160004B6579626F6172642073746172742E0AD8
:100170000055534220636F6E666967757265642E21
:100180000A000D0A696E69740A005B445D005B43F6
:100190005D001203480048004B00420020006D0043
:1001A0006F00640000000E0374002E006D002E002E
:1001B0006B002E0000000403090409028D000501F4
:1001C00000A032090400000103010100092111010E
:1001D00000012240000705810308000A090401000C
:1001E0000103010200092111010001224D00070550
:1001F000820308000A09040200010300000009212B
:10020000110100012236000705830308000A0904D2
:100210000300020300000009211101000122220055
:1002200007058403200001070504032000010904D9
:10023000040001030000000921110100012239001E
:10024000070585032000011201100100000008EDE0
:10025000FEFECA04010102000105010906A1010513
:100260000719E029E71500250195087501810205A8
:1002700008190129059505750191029501750391EC
:10028000010507190029F71500250195F875018169
:1002900002C00631FF0974A1010975150026FF008F
:1002A0009520750881020976150026FF00952075B6
:1002B000089102C005010980A1018502168100266E
:1002C000B7001A81002AB700751095018100C0059A
:1002D0000C0901A1018503160100269C021A0100E8
:1002E0002A9C02751095018100C005010902A10137
:1002F0000901A10005091901290515002501950528
:1003000075018102950175038101050109300931EB
:100310001581257F95027508810609381581257F8D
:10032000950175088106050C0A38021581257F950F
:100330000175088106C0C005010906A1010507195C
:10034000E029E715002501950875018102950175E1
:100350000881010508190129059505750191029586
:1003600001750391010507190029FF150026FF00FB
:10037000950675088100C0636F6E73756D65723A7E
:1003800020253034580A0073797374656D3A20253E
:100390003034580A000A002530325820006B657945
:1003A000626F6172643A20004C45443A2025303235
:1003B000580A00253032583A202530386225730A11
:1003C00000722F632030313233343536370A0064FF
:1003D000656C5F6B65795F6269743A2063616E2753
:1003E000742064656C3A20253032580A00616464D8
:1003F0005F6B65795F6269743A2063616E27742070
:100400006164643A20253032580A004F6E65736883
:100410006F743A2074696D656F75740A00290A005B
:100420002575002F002575005D280025640020003B
:10043000256400200025640020002564007C002540
:10044000303258006D6F7573656B6579205B62742F
:100450006E7C782079207620685D287265702F6127
:10046000636C293A205B006D6B5F776865656C5F34
:1004700074696D655F746F5F6D6178203D202564E0
:100480000A006D6B5F776865656C5F6D61785F739F
:1004900070656564203D2025640A006D6B5F74699A
:1004A0006D655F746F5F6D6178203D2025640A0083
:1004B0006D6B5F6D61785F7370656564203D2025AD
:1004C000640A006D6B5F696E74657276616C203DC5
:1004D0002025640A006D6B5F64656C6179203D20A6
:1004E00025640A006D6B5F776865656C5F74696D84
:1004F000655F746F5F6D6178203D2025640A006D33
:100500006B5F776865656C5F6D61785F737065655B
:1005100064203D2025640A006D6B5F74696D655F22
:10052000746F5F6D6178203D2025640A006D6B5FFC
:100530006D61785F7370656564203D2025640A00F5
:100540006D6B5F696E74657276616C203D20256409
:100550000A006D6B5F64656C6179203D2025640A3B
:10056000000A00257500363A20776865656C5F746F
:10057000696D655F746F5F6D61783A20000A0025D0
:100580007500353A20776865656C5F6D61785F73DB
:10059000706565643A20000A00257500343A2074BD
:1005A000696D655F746F5F6D61783A20000A0025A0
:1005B0007500333A206D61785F73706565643A2029
:1005C000000A00257500323A20696E746572766102
:1005D0006C286D73293A20000A00257500313A20F5
:1005E00064656C6179282A31306D73293A20000ADC
:1005F000092D2056616C756573202D0A004D3E0053
:100600004D25643E20003F0073657420646566617B
:10061000756C740A00433E2000776865726520643B
:10062000656C74613A20637572736F723D25642C3A
:1006300020776865656C3D25640A5365652068749C
:1006400074703A2F2F656E2E77696B6970656469D7
:10065000612E6F72672F77696B692F4D6F757365A8
:100660005F6B6579730A000A092D204D6F757365FC
:100670006B6579202D0A4553432F713A09717569CD
:10068000740A313A0964656C6179282A31306D73D6
:10069000290A323A09696E74657276616C286D7345
:1006A000290A333A096D61785F73706565640A34AD
:1006B0003A0974696D655F746F5F6D61780A353AE8
:1006C00009776865656C5F6D61785F7370656564F7
:1006D0000A363A09776865656C5F74696D655F74A1
:1006E0006F5F6D61780A0A703A097072696E7420E2
:1006F00076616C7565730A643A0973657420646584
:100700006661756C74730A75703A092B310A646FEF
:10071000776E3A092D310A706775703A092B3130BE
:100720000A7067646F776E3A092D31300A0A737068
:10073000656564203D2064656C7461202A206D61CC
:10074000785F7370656564202A2028726570656122
:1007500074202F2074696D655F746F5F6D617829F7
:100760000A003F004D3E2000433E20004C25640A15
:10077000000A092D20436F6E736F6C65202D0A45AA
:1007800053432F713A09717569740A6D3A096D6F97
:100790007573656B65790A000A092D204D616769DB
:1007A00063202D0A643A0964656275670A783A091C
:1007B0006465627567206D61747269780A6B3A09C5
:1007C0006465627567206B6579626F6172640A6D3A
:1007D0003A096465627567206D6F7573650A763ACC
:1007E0000976657273696F6E0A733A09737461747E
:1007F00075730A633A09636F6E736F6C65206D6F72
:1008000064650A302D343A096C61796572302D3493
:10081000284631302D4634290A506175733A0962F1
:100820006F6F746C6F616465720A6E3A094E4B5259
:100830004F0A003F004E4B524F3A206F66660A0047
:100840004E4B524F3A206F6E0A0074696D65725FAD
:1008500072656164333228293A202530346C580A95
:10086000006B6579626F6172645F6E6B726F3A20C4
:1008700025580A006B6579626F6172645F69646C08
:10088000653A2025580A006B6579626F6172645F72
:1008900070726F746F636F6C3A2025580A00686F2E
:1008A00073745F6B6579626F6172645F6C656473AA
:1008B00028293A2025580A000A092D20537461740A
:1008C0007573202D0A004743433A20342E392E32C7
:1008D000204156522D4C4942433A20312E382E3079
:1008E00073766E204156525F415243483A206176FA
:1008F00072350A004F5054494F4E533A204C5546DA
:1009000041204D4F5553454B455920455854524170
:100910004B455920434F4E534F4C4520434F4D4D6F
:10092000414E44204E4B524F204B45594D41505F54
:1009300053454354494F4E20343039360A0042550E
:10094000494C443A20343139303537312D6469729D
:100950007479202830373A35353A3435204F63746E
:100960002032382032303137290A005649443A20A3
:1009700030784645454428742E6D2E6B2E29205024
:1009800049443A203078434146452848484B422064
:100990006D6F6429205645523A203078303130341A
:1009A0000A00444553433A20742E6D2E6B2E206B63
:1009B0006579626F617264206669726D77617265D4
:1009C00020666F722048484B42206D6F640A000A0F
:1009D000092D2056657273696F6E202D0A000A6D0D
:1009E0006F7573653A206F66660A000A6D6F7573DE
:1009F000653A206F6E0A000A6B6579626F617264F6
:100A00003A206F66660A000A6B6579626F617264EC
:100A10003A206F6E0A000A6D61747269783A206F2D
:100A200066660A000A6D61747269783A206F6E0A10
:100A3000000A64656275673A206F6E0A000A646591
:100A40006275673A206F66660A000A0A626F6F7401
:100A50006C6F616465722E2E2E2000433E200000D4
:100A600011241FBECFEFDAE0DEBFCDBF04B603FE18
:100A700027C08091A2029091A302A091A402B091FC
:100A8000A5028730904BA740B04BD1F41092A20240
:100A90001092A3021092A4021092A50214BE84B771
:100AA000877F84BF0FB6F894A89580916000886115
:100AB00080936000109260000FBEE0E0F8E30995BB
:100AC00011E0A0E0B1E0EAE1FBE402C005900D9284
:100AD000A833B107D9F722E0A8E3B1E001C01D9225
:100AE000A23AB207E1F70E94C1090C948B250C943D
:100AF0000000FF93EF93E0913801F09139013097B6
:100B000009F00995EF91FF910895FC0185918030DE
:100B100011F0EFDFFBCF0895FF27E0E230E247FF5F
:100B20000CC0419597FF09C0EDE2609570958095E6
:100B30009095611D711D811D911D27FF02C021959A
:100B400030E350E2AA27660F771F881F991FAA1F5C
:100B5000A41710F0A41B63955A95A9F7AA3008F0C2
:100B6000A95FA05DAF93F3956115710581059105AE
:100B700041F7ED3211F4EF93F395F21718F43F9328
:100B8000F395FBCF8F91B5DFFA95E1F70895E991E1
:100B9000F9918591803021F0853219F0AADFF9CFE3
:100BA000089520E0E89455915532C1F3503311F483
:100BB000689455915A3348F4505390F3220F022E03
:100BC000220F220F200D250FF4CF0EF421958991CD
:100BD0009991533619F3533729F1533559F1BC0123
:100BE00088279927E8945C3621F489919991689433
:100BF0005591543639F446EF7EF077FF0DC08FEFF4
:100C00009FEF0AC055374AE039F0583540E121F0EE
:100C1000523642E009F00895FF93EF937DDFEF91A4
:100C2000FF91B7CFFF93EF93FC0181918030B9F32F
:100C300060DFFBCFFF93EF9368DFF1CFDF93CF93BC
:100C4000CDB7DEB72596A3DFCF91DF9108958FEF63
:100C500084B980E485B957985F9A87B1806C87B969
:100C600088B1806C88B92E9A2F98EAE4F1E080E18F
:100C70008E0F11928E13FDCFEAE3F1E080E18E0F2B
:100C800011928E13FDCF8AE491E090935D018093E1
:100C90005C018AE391E090935B0180935A0108958F
:100CA000EF92FF920F931F93CF93DF9380915A019E
:100CB00090915B0120915C0130915D0130935B016B
:100CC00020935A0190935D0180935C01C0E0D0E0D5
:100CD00001E010E080E090E0FC2FF770EC2FE8706E
:100CE00025B1207C2F2BAC0133E0440F551F3A95E2
:100CF000E1F7242B25B928B12F73EE2311F02064DE
:100D000001C0206828B92AE12A95F1F700C0A09116
:100D10005A01B0915B01AC0FBD1F2C9130E0082E41
:100D200002C0359527950A94E2F720FD2F9AA5E396
:100D3000AA95F1F70000F6B42E98BAE1BA95F1F74A
:100D400000C040915C0150915D01BA016C0F7D1FA4
:100D50004F9B0BC09801082E01C0220F0A94EAF79E
:100D60002095DB013C91232309C0DB01EC90980125
:100D7000082E01C0220F0A94EAF72E292C9326B5DB
:100D80006F2D70E02F1518F026B530E004C026B5A1
:100D900030E021503F4F261B370B2630310558F0ED
:100DA000A0915A01B0915B01AC0FBD1F2C91DA01EB
:100DB000AC0FBD1F2C93BAE1BA95F1F700C02F9884
:100DC0002E9A20EA2A95F1F701968830910509F0CC
:100DD00087CFA0915C01B0915D01AC0FBD1FE09188
:100DE0005A01F0915B01EC0FFD1F9C9180819817D7
:100DF00051F00E94A01C60935E0170935F0180938C
:100E00006001909361012196C031D10509F062CF54
:100E100080919902853021F080919902811111C051
:100E200060915E0170915F0180916001909161011C
:100E30000E94D61C613177428105910510F00E9415
:100E4000211C81E0DF91CF911F910F91FF90EF90D6
:100E5000089520915C0130915D01F901E80FF11DC9
:100E60008081089508950895569A81FF02C05E9A80
:100E700008955E9808958091860108959FB7F8942B
:100E8000109265019FBF90919902943009F057C06C
:100E90009091E9009F703091EC00232F217030FD7C
:100EA00020E8922B24E02093E9002091EB0020FF22
:100EB00043C02091EE0027FF3FC020916201222312
:100EC00021F02091E80025FF37C01092620126E052
:100ED0003091E80035FD15C030919902343061F54C
:100EE0003091EB0035FD28C0215021F481E0809342
:100EF000620122C0EFE9FFE03197F1F700C0000086
:100F0000E7CF8093F1008091E80085FD0AC08091D1
:100F1000E80080FFFCCF8091E8008E778093E800A6
:100F200006C08FB7F89421E0209365018FBF9F70B2
:100F30009093E90080E008959F709093E9008FEF0F
:100F40000895CF93DF9300D01F92CDB7DEB79C01F9
:100F500080919902843019F593E099833B832A8329
:100F60009093E9008FEF9091E800815095FD06C0C5
:100F700095ED9A95F1F700008111F5CF8091E80089
:100F800085FF0DC040E050E063E070E0CE010196C7
:100F90000E94830A8091E8008E778093E8000F908A
:100FA0000F900F90DF91CF910895CF93DF9300D0F2
:100FB0001F92CDB7DEB720919902243021F522E0AF
:100FC00029839B838A8383E08093E9008FEF90914C
:100FD000E800815095FD06C095ED9A95F1F7000067
:100FE0008111F5CF8091E80085FF0DC040E050E011
:100FF00063E070E0CE0101960E94830A8091E800D0
:101000008E778093E8000F900F900F90DF91CF9133
:101010000895209199022430F1F422E02093E90010
:101020002FEF3091E800215035FD06C035ED3A959F
:10103000F1F700002111F5CF2091E80025FF0BC04A
:1010400040E050E065E070E00E94830A8091E80093
:101050008E778093E8000895CF93DF9320919902D3
:10106000243009F048C0EC0180910A018823E1F0A6
:1010700080910B018823C1F085E08093E9008FEF18
:101080009091E800815095FD06C09AE29A95F1F79B
:1010900000C08111F5CF8091E80085FF2CC040E0B1
:1010A00050E060E270E017C081E08093E9008FEFCC
:1010B0009091E800815095FD06C095ED9A95F1F765
:1010C00000008111F5CF8091E80085FF14C040E059
:1010D00050E068E070E0CE010E94830A8091E80051
:1010E0008E778093E80080E2FE01A6E6B1E00190F1
:1010F0000D928A95E1F7DF91CF9108958EE891E006
:101100000E94850580919802811109C00E94180CE7
:101110000E94750C8091E20084608093E200089543
:101120008AE891E00E94850510929802089508953A
:10113000209163012F5F822F62E30E945125992342
:1011400019F0209363010895109263018091650165
:10115000882371F180919902843041F58091E900F2
:101160008F702091EC00922F917020FD90E8892BD8
:1011700094E09093E9009091EB0090FF14C090915F
:10118000EE0097FF10C09091E80095FF03C0109209
:10119000F100F9CF9091E80090FF05C09091E80030
:1011A0009E779093E8008F708093E900109265011C
:1011B000089542E061EC81E00E94920B42E061EC14
:1011C00082E00E94920B42E061EC83E00E94920B6D
:1011D00042E261EC84E00E94920B42E261EC85E025
:1011E0000C94920B80919B02833009F455C030F42B
:1011F000813071F0823009F48EC008958A3009F48C
:101200007AC08B3009F460C0893009F09CC020C0DE
:1012100080919A02813A09F096C08091E800877F18
:101220008093E80080919E0290919F02892B21F487
:1012300060E286E691E003C060E080E090E070E06C
:101240000E94CE0A8091E8008B778093E800089591
:1012500080919A02813209F076C080919E0290912D
:101260009F02009719F0049709F06DC08091E80083
:10127000877F8093E8008091E80082FD05C080911F
:1012800099028111F8CF5FC08091F10080938601AF
:101290008091E8008B7753C080919A02813A09F0DF
:1012A00052C080919E0290919F02892B09F04BC001
:1012B0008091E800877F8093E8008091E80080FFBC
:1012C000FCCF80910A0136C080919A028132D9F513
:1012D00080919E0290919F02892BA9F58091E80050
:1012E000877F8093E8000E94C70B80919C028093C7
:1012F0000A010C94F11480919A02813221F58091B7
:10130000E800877F8093E8000E94C70B80919D02D0
:1013100080938701089580919A02813AA1F4809187
:10132000E800877F8093E8008091E80080FFFCCF91
:10133000809187018093F1008091E8008E778093FF
:10134000E8000C94C70B08950895089580918601D4
:10135000809364011092860180E00E9434070E940D
:101360008E100C94F1140C94A6090E94211C8091FB
:101370009702882329F00E944A1C81110C946D0A5F
:10138000089584B7877F84BF0FB6F894A89580919D
:101390006000886180936000109260000FBE90E052
:1013A00080E80FB6F89480936100909361000FBEBF
:1013B0008EE397E00E94F21B82E891E00E9485058F
:1013C0000E94A4090E94BB0F0E94180C0E94750C79
:1013D0008091E20084608093E20078948091990289
:1013E0008430E1F781E791E00E9485050E94BD0FFE
:1013F00080E091E00E94FA0E80E691E00E9485056F
:101400000E94A50980919902853019F40E94B509BE
:10141000F9CF0E94C10FF6CF0E945E1C809164013B
:101420008093860108950C940C0A292F33272330CA
:101430003105C9F064F42130310581F022303105E5
:1014400009F043C08DE890E02AEB31E042C0213240
:101450003105F1F02232310541F137C082E190E0EF
:1014600027E432E036C099278130910541F082307F
:10147000910541F0892B49F5E6EBF1E005C0E6EA7C
:10148000F1E002C0E2E9F1E0849190E09F0121C027
:101490006530D8F4E62FF0E0EE0FFF1FED5DFE4F54
:1014A0002081318189E090E014C0653070F470E0F3
:1014B000FB01EE0FFF1FE75EFE4F20813181FB0134
:1014C000EC5EFE4F808190E004C080E090E020E080
:1014D00030E0FA0131832083089580E189BD82E103
:1014E00089BD09B400FEFDCF8091D8008F7D809327
:1014F000D8008091E00082608093E0008091E0005D
:1015000081FDFCCF0895CF92DF92EF92FF920F936F
:101510001F93CF93DF93EC018B016A010E94E60BCE
:10152000811133C0C114D10439F0F6018081918159
:10153000081B190BC80FD91FE12CF12C011511053F
:1015400019F18091E80085FD16C08091E8008E7742
:101550008093E800C114D10449F0F60180819181A3
:10156000E80EF91EF182E08285E00FC00E94E60BD2
:10157000882321F30AC089918093F1000150110959
:10158000FFEFEF1AFF0ADACF80E0DF91CF911F91D2
:101590000F91FF90EF90DF90CF9008952091A002DF
:1015A0003091A1022617370748F06115710539F40B
:1015B0002091E8002E772093E80001C0B90140E0B7
:1015C00061157105A9F120919902222309F443C004
:1015D000253009F442C02091E80023FD40C020914D
:1015E000E80022FD32C02091E80020FFE9CF4091C1
:1015F000F3002091F20030E0342BFC01CF016115A3
:10160000710559F02830310540F481918093F10043
:10161000615071092F5F3F4FF1CF41E02830310514
:1016200009F040E02091E8002E772093E800C8CF31
:101630004111C9CF0AC080919902882361F0853099
:1016400061F08091E80083FD0AC08091E80082FF8C
:10165000F2CF80E0089582E0089583E0089581E06C
:1016600008952091A0023091A1022617370748F073
:101670006115710539F42091E8002E772093E80078
:1016800001C0B901FC0120E06115710591F1809163
:101690009902882309F440C0853009F43FC0809145
:1016A000E80083FD3DC08091E80082FD2FC080915D
:1016B000E80080FFE9CF2091F3008091F20090E0F4
:1016C000922B6115710559F08830910540F42491F1
:1016D0002093F1003196615071090196F2CF21E01B
:1016E000089709F020E08091E8008E778093E80069
:1016F000CBCF2111CCCF0AC080919902882361F011
:10170000853061F08091E80083FD0AC08091E80097
:1017100082FFF2CF80E0089582E0089583E008958B
:1017200081E00895982F973058F59093E900981725
:1017300039F07091EC002091ED005091F00003C061
:10174000242F762F50E021FF19C03091EB003E7F0F
:101750003093EB003091ED003D7F3093ED00309100
:10176000EB0031603093EB007093EC002093ED00C0
:101770005093F0002091EE0027FF07C09F5FD3CF6A
:101780008F708093E90081E0089580E00895809152
:101790009A0287FF11C08091E80082FD05C0809108
:1017A00099028111F8CF11C08091E8008B770BC0AE
:1017B00080919902882349F08091E80080FFF8CF5A
:1017C0008091E8008E778093E80008952091E400EE
:1017D0003091E50095E64091EC00842F817040FF48
:1017E00022C08091E80080FD1CC08091990288236E
:1017F00091F0853091F08091EB0085FD10C0409113
:10180000E4005091E5004217530729F39A019150E3
:1018100011F784E0089582E0089583E0089581E05F
:10182000089580E008954091E80042FFDECF0895DA
:101830000E94860C0E948E0CE0EEF0E080818160B8
:101840008083E8EDF0E080818F77808319BCA7ED7D
:10185000B0E08C918E7F8C9380818F7E80831092FC
:10186000980208950F931F93CF93DF930E94860CE5
:101870000E948E0CC8EDD0E088818F7788838881A4
:101880008068888388818F7D888319BC1092990233
:1018900010929502109297021092960200EE10E0BC
:1018A000F80180818B7F808388818160888342E01A
:1018B00060E080E00E94920BE1EEF0E080818E7F9C
:1018C0008083E2EEF0E080818160808380818860A7
:1018D0008083F80180818E7F808388818061888306
:1018E000DF91CF911F910F910895E8EDF0E0808195
:1018F0008F7E8083E7EDF0E080818160808384E0EB
:1019000082BF81E0809398020C94320CE8EDF0E005
:1019100080818E7F80831092E20008951092DA0019
:101920001092E10008951F920F920FB60F921124AA
:101930002F933F934F935F936F937F938F939F93D7
:10194000AF93BF93EF93FF938091E10082FF0BC0B1
:101950008091E20082FF07C08091E1008B7F80933D
:10196000E1000E9498088091DA0080FF1FC08091FA
:10197000D80080FF1BC08091DA008E7F8093DA0050
:101980008091D90080FF0DC080E189BD82E189BDD1
:1019900009B400FEFDCF81E0809399020E947E0889
:1019A00005C019BC109299020E9490088091E10034
:1019B00080FF19C08091E20080FF15C08091E20095
:1019C0008E7F8093E2008091E20080618093E2004C
:1019D0008091D80080628093D80019BC85E0809304
:1019E00099020E94B3098091E10084FF30C0809188
:1019F000E20084FF2CC080E189BD82E189BD09B489
:101A000000FEFDCF8091D8008F7D8093D80080911B
:101A1000E1008F7E8093E1008091E2008F7E8093D1
:101A2000E2008091E20081608093E2008091950263
:101A3000882311F084E007C08091E30087FD02C095
:101A400081E001C083E0809399020E94130A809193
:101A5000E10083FF29C08091E20083FF25C08091CF
:101A6000E100877F8093E10082E0809399021092E9
:101A700095028091E1008E7F8093E1008091E200E9
:101A80008E7F8093E2008091E20080618093E2008B
:101A900042E060E080E00E94920B8091F00088605C
:101AA0008093F0000E949708FF91EF91BF91AF9152
:101AB0009F918F917F916F915F914F913F912F9166
:101AC0000F900FBE0F901F9018951F920F920FB698
:101AD0000F9211242F933F934F935F936F937F93B4
:101AE0008F939F93AF93BF93CF93DF93EF93FF9326
:101AF000C091E900CF708091EC00D82FD17080FDAB
:101B0000D0E81092E9008091F000877F8093F00088
:101B100078940E94A90D1092E9008091F0008860ED
:101B20008093F000CD2BCF70C093E900FF91EF912F
:101B3000DF91CF91BF91AF919F918F917F916F91E5
:101B40005F914F913F912F910F900FBE0F901F907B
:101B500018951F93CF93DF93CDB7DEB7AA970FB633
:101B6000F894DEBF0FBECDBFEAE9F2E088E08E0F49
:101B70009091F10091938E13FBCF0E94F208809117
:101B8000E80083FF1FC180919A0290919B02492F28
:101B900050E04A30510508F015C1FA01EA5AFF4FEA
:101BA0000C947125803881F0823809F00BC1809146
:101BB0009E028F708093E9008091EB0085FB88275F
:101BC00080F91092E90006C08091960290919702E8
:101BD000911182609091E800977F9093E800809344
:101BE000F1001092F100C8C0282F2D7F09F0EAC043
:101BF000882319F0823061F0E5C080919C02813029
:101C000009F0E0C0933009F080E0809397022BC088
:101C100080919C02811127C080919E028F7009F4EF
:101C2000D1C08093E9002091EB0020FF1CC09330CD
:101C300021F48091EB00806214C09091EB009061E0
:101C40009093EB0021E030E0A90102C0440F551F42
:101C50008A95E2F74093EA001092EA008091EB0047
:101C600088608093EB001092E9008091E800877F04
:101C700086C08111A7C010919C021F778091E3005C
:101C80008078812B8093E3008091E800877F8093A8
:101C9000E8000E94C70B8091E80080FFFCCF809194
:101CA000E30080688093E300111102C082E001C06C
:101CB00083E08093990286C08058823008F082C009
:101CC00080919C0290919D028C3D53E0950779F59F
:101CD00083E08A838AE289834FB7F894DE01139602
:101CE00020E03EE051E2E32FF0E050935700E49112
:101CF00020FF03C0E295EF703F5FEF708E2F90E002
:101D0000EA3010F0C79601C0C0968D939D932F5F67
:101D1000243149F74FBF8091E800877F8093E80026
:101D20006AE270E0CE0101960E94CE0A14C0AE01B4
:101D30004F5F5F4F60919E020E94150ABC01892B84
:101D400009F440C09091E800977F9093E800898162
:101D50009A810E94310B8091E8008B778093E80094
:101D600031C0803879F58091E800877F8093E80062
:101D7000809195028093F1008091E8008E778093A6
:101D8000E8000E94C70B1EC081111CC090919C02EC
:101D90009230C0F48091E800877F8093E8009093B0
:101DA00095020E94C70B80919502811106C0809117
:101DB000E30087FD02C081E001C084E080939902C6
:101DC0000E94D9088091E80083FF0AC08091E80052
:101DD000877F8093E8008091EB0080628093EB0026
:101DE000AA960FB6F894DEBF0FBECDBFDF91CF919C
:101DF0001F91089590938D0180938C010895E09137
:101E00008C01F0918D01309721F00190F081E02D4F
:101E1000099480E00895EF92FF920F931F93CF9360
:101E2000DF93E0918C01F0918D013097B1F18C013D
:101E30000280F381E02D09958091840282FF2DC0FC
:101E400080FF04C08DE993E00E948505E80110E25F
:101E500087E9E82E83E0F82E8091840280FF0BC092
:101E600088811F928F93FF92EF920E941E060F901F
:101E70000F900F900F90115021961111EDCF80917E
:101E8000840280FF0AC085E993E0DF91CF911F9122
:101E90000F91FF90EF900C948505DF91CF911F91EA
:101EA0000F91FF90EF900895E0918C01F0918D01DA
:101EB000309721F00480F581E02D09940895CF93A7
:101EC000DF93EC0180918A0190918B01C817D907AB
:101ED00009F1D0938B01C0938A01E0918C01F091BC
:101EE0008D013097B9F00680F781E02DCE0109957C
:101EF0008091840282FF0EC080FF0CC0DF93CF93DD
:101F000087E893E09F938F930E941E060F900F9097
:101F10000F900F90DF91CF910895CF93DF93EC0155
:101F20008091880190918901C817D90709F1D09350
:101F30008901C0938801E0918C01F0918D01309767
:101F4000B9F00084F185E02DCE01099580918402DD
:101F500082FF0EC080FF0CC0DF93CF9387E793E032
:101F60009F938F930E941E060F900F900F900F90DB
:101F7000DF91CF9108950C948F100E948B1C0C94CC
:101F800027065F926F927F928F929F92AF92BF923D
:101F9000CF92DF92EF92FF920F931F93CF93DF9335
:101FA00000D000D01F92CDB7DEB70E9450068FE858
:101FB000C82E81E0D82E512C88248394912C852D15
:101FC0000E942907A82EF601E080E82641F45394E8
:101FD000FFEFCF1ADF0A80E15812F1CF40C08091A5
:101FE000840281FD0E94901000E010E0F12CB12CE1
:101FF000C701002E02C0959587950A94E2F780FFED
:1020000028C009835A823401002E02C0660C771C56
:102010000A94E2F793012A213B2181E0232B09F462
:1020200080E08B830E94941C8160782F9D838C8339
:1020300049815A816B818D810E94C41049815A81E6
:102040006B817C818D810E940E1CF6018081682647
:1020500060820F5F1F4F0830110551F6B8CF8FEF28
:1020600089838A831B820E94941C8160782F9D83C0
:102070008C8349815A816B818D810E94C4100E949A
:102080000D1C0E94811F10918E010E94FF0E1817D7
:1020900071F10E94FF0E80938E019091840292FF55
:1020A0000EC090FF0CC01F928F9388EA93E09F931D
:1020B0008F930E941E060F900F900F900F908091AB
:1020C0008E010F900F900F900F900F90DF91CF9196
:1020D0001F910F91FF90EF90DF90CF90BF90AF9046
:1020E0009F908F907F906F905F900C941F1C0F902B
:1020F0000F900F900F900F90DF91CF911F910F9144
:10210000FF90EF90DF90CF90BF90AF909F908F9017
:102110007F906F905F9008950C9434070895089510
:10212000EF92FF920F931F93CF93DF9381EC93E095
:102130000E948505C0E0D0E08DE2E82E81E0F82E17
:1021400003EB13E08C2F0E9429070E94F71BFF92DC
:10215000EF921F928F93DF93CF931F930F930E9461
:102160001E0621968DB79EB708960FB6F8949EBFAF
:102170000FBE8DBFC031D10529F7DF91CF911F91DF
:102180000F91FF90EF900895CF93DF93CDB7DEB717
:102190002B970FB6F894DEBF0FBECDBF942F4F83A1
:1021A000252F588769877A878B874A855B85452BDA
:1021B00021F02F3F09F59F3FF9F4DE01119686E0EB
:1021C000FD0111928A95E9F785E0FE0137960190AD
:1021D0000D928A95E1F749815A816B817C818D81CD
:1021E0009E810E94D6172B960FB6F894DEBF0FBEC5
:1021F000CDBFDF91CF9108954F81588569857A854C
:102200008B850E940E1CD9CFCF93882309F465C01B
:10221000C82F8CEF8C0F813A20F080E58C0F8E3226
:1022200048F48C2F0E94CB22811157C08C2F0E9422
:10223000AE1A0CC080E28C0F883058F4C77081E071
:1022400001C0880FCA95EAF70E94591BCF910C94E0
:102250009D1B8BE58C0F833078F4C53A29F0C63A84
:1022600031F083E890E005C081E890E002C082E8A8
:1022700090E0CF910C945F0F88E58C0F853168F565
:10228000C83A89F0C93A91F0CA3A99F0CB3AA1F02C
:10229000CC3AA9F0CD3AB1F0CE3AB9F0CF3AC1F08C
:1022A00080E090E017C082EE90E014C089EE90E0EC
:1022B00011C08AEE90E00EC085EB90E00BC086EB7B
:1022C00090E008C083EB90E005C084EB90E002C092
:1022D00087EB90E0CF910C948D0FCF9108958823D8
:1022E00049F19CEF980F913A20F090E5980F9E32BB
:1022F00018F40E94011B0DC090E2980F983058F41A
:10230000877091E001C0990F8A95EAF7892F0E94A2
:102310005F1B0C949D1B9BE5980F933020F480E08D
:1023200090E00C945F0F885A853120F480E090E0B3
:102330000C948D0F0895882321F00E94591B0C9452
:102340009D1B0895882321F00E945F1B0C949D1B08
:102350000895BF92CF92DF92EF92FF920F931F9357
:10236000CF93DF9300D000D000D0CDB7DEB725E00B
:10237000FC01DE01119601900D922A95E1F7FC0116
:1023800040815181028163817481258122952F7062
:102390006115710509F403C35F3F19F44F3F09F458
:1023A000FEC26C01862F7D836C83602F782F8D8118
:1023B0002E830E94321A182FB92E0E94311A0E94C1
:1023C0002119EB2DE295EF70F0E0E05AFF4F2E81DE
:1023D0000C9471258B2D807F9B2D9F70F92E882367
:1023E00019F0F29490EFF922002349F0FF2009F44C
:1023F00083C28F2D0E946C1B0E949D1B7DC2812F6A
:102400000E946F11FF2009F4CAC28F2D0E94721B17
:1024100026960FB6F894DEBF0FBECDBFDF91CF91E9
:102420001F910F91FF90EF90DF90CF90BF900C9491
:102430009D1B8B2D807F9B2D9F70F92E803219F074
:10244000F29480EFF822112319F0113009F12AC01B
:102450000023B1F08F2D222351F1213041F5269632
:102460000FB6F894DEBF0FBECDBFDF91CF911F91A5
:102470000F91FF90EF90DF90CF90BF900C947C1B5A
:10248000222319F0213009F48AC20E94851B2DC035
:102490000023F1F0263008F082C20E94561B8F21E3
:1024A00029F023C00023F9F0211116C08F2D2696A4
:1024B0000FB6F894DEBF0FBECDBFDF91CF911F9155
:1024C0000F91FF90EF90DF90CF90BF900C949B11F5
:1024D000253008F064C209C0F601858180FF0CC276
:1024E0008F708583E3CF21111CC28F2D83C12B2DCB
:1024F00026952695237030E02115310521F02130F5
:102500003105D1F04CC2002321F0812F9B2D937017
:1025100002C080E090E026960FB6F894DEBF0FBEB2
:10252000CDBFDF91CF911F910F91FF90EF90DF9082
:10253000CF90BF900C945F0F002321F0812F9B2D33
:10254000937002C080E090E026960FB6F894DEBF4C
:102550000FBECDBFDF91CF911F910F91FF90EF90F4
:10256000DF90CF90BF900C948D0F812F002319F036
:102570000E94071E02C00E946F1E26960FB6F89496
:10258000DEBF0FBECDBFDF91CF911F910F91FF90A6
:10259000EF90DF90CF90BF900C94F41E8B2D837042
:1025A00009F07BC00111FBC1812F82958695877050
:1025B000880F880F912F9F70C92ED12CE12CF12C00
:1025C000082E04C0CC0CDD1CEE1CFF1C0A94D2F7B4
:1025D00014FF12C04FE050E060E070E004C0440F10
:1025E000551F661F771F8A95D2F7CB01BA016095F8
:1025F00070958095909503C060E070E0CB012B2D25
:10260000269526952370422F50E042305105D9F08F
:102610004330510569F16C297D298E299F2941306C
:10262000510551F126960FB6F894DEBF0FBECDBF0F
:10263000DF91CF911F910F91FF90EF90DF90CF909E
:10264000BF900C9446196C297D298E299F292696C6
:102650000FB6F894DEBF0FBECDBFDF91CF911F91B3
:102660000F91FF90EF90DF90CF90BF900C94601986
:102670000E944619C701B60126960FB6F894DEBF30
:102680000FBECDBFDF91CF911F910F91FF90EF90C3
:10269000DF90CF90BF900C942C19002319F08B2D54
:1026A000817001C08695882309F479C1812F8295B4
:1026B00086958770880F880F912F9F70C92ED12C17
:1026C000E12CF12C082E04C0CC0CDD1CEE1CFF1CF0
:1026D0000A94D2F714FF12C04FE050E060E070E0BF
:1026E00004C0440F551F661F771F8A95D2F7CB0190
:1026F000BA01609570958095909503C060E070E098
:10270000CB012B2D269526952370422F50E0423089
:102710005105D9F04330510569F16C297D298E2985
:102720009F294130510551F126960FB6F894DEBF2E
:102730000FBECDBFDF91CF911F910F91FF90EF9012
:10274000DF90CF90BF900C940D1A6C297D298E29B3
:102750009F2926960FB6F894DEBF0FBECDBFDF913E
:10276000CF911F910F91FF90EF90DF90CF90BF908E
:102770000C941F1A0E940D1AC701B60126960FB6B7
:10278000F894DEBF0FBECDBFDF91CF911F910F91A7
:10279000FF90EF90DF90CF90BF900C94FB19103F0B
:1027A000D1F128F480E4810F803250F0A0C0123FB4
:1027B00009F462C008F44BC0133F09F472C097C01B
:1027C000F12FF071FF2E8B2D8F71002351F00E949D
:1027D0009419812FFF2019F08295807F68CE8F7029
:1027E00066CE0E94B519812FFF2019F08295807F57
:1027F00001C08F7026960FB6F894DEBF0FBECDBF16
:10280000DF91CF911F910F91FF90EF90DF90CF90CC
:10281000BF900C94A2110023B1F0253008F0BFC086
:102820008B2D8F7126960FB6F894DEBF0FBECDBFED
:10283000DF91CF911F910F91FF90EF90DF90CF909C
:10284000BF900C94DA19263008F0A9C0E9CF002314
:10285000A9F08B2D8F7126960FB6F894DEBF0FBEB0
:10286000CDBFDF91CF911F910F91FF90EF90DF903F
:10287000CF90BF900C949419002359F38B2D8F7136
:1028800026960FB6F894DEBF0FBECDBFDF91CF9175
:102890001F910F91FF90EF90DF90CF90BF900C941D
:1028A000B519002399F08B2D8F7126960FB6F894E9
:1028B000DEBF0FBECDBFDF91CF911F910F91FF9073
:1028C000EF90DF90CF90BF900C947F1926960FB6B3
:1028D000F894DEBF0FBECDBFDF91CF911F910F9156
:1028E000FF90EF90DF90CF90BF900C947A19002367
:1028F000A9F0222309F4ADCF812F26960FB6F894C4
:10290000DEBF0FBECDBFDF91CF911F910F91FF9022
:10291000EF90DF90CF90BF900C940411222309F424
:10292000ADCF812F26960FB6F894DEBF0FBECDBF78
:10293000DF91CF911F910F91FF90EF90DF90CF909B
:10294000BF900C946F114B2D4F70612FC6010E94E8
:10295000811D26960FB6F894DEBF0FBECDBFDF9166
:10296000CF911F910F91FF90EF90DF90CF90BF908C
:102970000C947A184B2D4F70612FC60126960FB616
:10298000F894DEBF0FBECDBFDF91CF911F910F91A5
:10299000FF90EF90DF90CF90BF900C94841D26960F
:1029A0000FB6F894DEBF0FBECDBFDF91CF911F9160
:1029B0000F91FF90EF90DF90CF90BF9008950E940D
:1029C000791B0E94481B0E949D1B0E9426200E948A
:1029D000F41E80E090E00E945F0F80E090E00C9495
:1029E0008D0F0E94691B0C94DF14CF93DF9300D0EE
:1029F00000D01F92CDB7DEB7942F4983252F5A837D
:102A00006B837C838D834C815D81452B39F12F3F16
:102A100011F49F3F19F149815A816B817C818D812D
:102A20000E94321A292F22952F7030E02C30310568
:102A300004F52A3031055CF4225031092230310589
:102A400068F4853A80F4843090F4823080F0883ED7
:102A500038F4803E60F48450813A48F080E014C03D
:102A6000803FE1F704C090E2980F983080F781E052
:102A70000BC02C30310521F493FB882780F904C06A
:102A80002F303105C9F3EACF0F900F900F900F90C0
:102A90000F90DF91CF910895CF93DF9300D000D0B6
:102AA0001F92CDB7DEB70F900F900F900F900F9041
:102AB000DF91CF910895CF93DF9300D000D000D065
:102AC000CDB7DEB726960FB6F894DEBF0FBECDBFEA
:102AD000DF91CF9108951F93CF93DF93C0919F0112
:102AE00016E08091A001C81799F0D0E01C9FF0017A
:102AF0001D9FF00D1124EF55FE4F408151816281E1
:102B00007381848195810E945B152196C770E9CFFE
:102B1000DF91CF911F9108954091D1015091D20141
:102B20006091D3017091D4018091D5019091D6012B
:102B30000C945B158091D60182958F7009F054C07A
:102B40008091D301882309F44FC080919F01A09107
:102B5000A0016091D1017091D2014091D4015091B6
:102B6000D501B6E08A1709F43FC090E04115510540
:102B7000C1F17F3F11F46F3FA1F1B89FF001B99F00
:102B8000F00D1124EF55FE4F218172132AC02081D0
:102B9000621327C02281211124C02381348124178C
:102BA000350710F421503109241B350B2C323140EC
:102BB000C0F42091D6012F7020612093D60126E029
:102BC000289FF001299FF00D1124EA55FE4F8081C6
:102BD0008F708061808381ED91E00E94A9110C9437
:102BE0006B1501968770BECF0895BF92CF92DF928A
:102BF000EF92FF920F931F93CF93DF93CDB7DEB782
:102C000061970FB6F894DEBF0FBECDBF7C0185E0A3
:102C1000F701DE011D9601900D928A95E1F7D7012B
:102C20004C9111965C9111971296DC901297139625
:102C30000D911C9114973091D1016091D201809136
:102C4000D4019091D501009709F47FC16F3F19F429
:102C50003F3F09F47AC1B090D301BB2009F4CAC048
:102C60002091D6010817190750F0F801E81BF90B5D
:102C7000CF01CC24C3948C329140D0F009C0809510
:102C80009095800F911FCC24C3948C32914080F09A
:102C9000C12C207F09F0CCC0702F198B088B6D2DB3
:102CA00089890E944C1581ED91E00E94A911B6C05E
:102CB000822F807F09F047C0651314C0341312C0FF
:102CC000D11010C02F7020612093D6010E948C1566
:102CD00081ED91E00E94A9118091D601D70115964E
:102CE0008C932FC00115110519F15F3F11F44F3F6F
:102CF000F9F0CD2CD1101CC080919F012091A00132
:102D000036E0821709F45CC090E0389FF001399FEB
:102D1000F00D1124EF55FE4F6181561306C06081FE
:102D2000461303C06281611103C001968770E9CF29
:102D3000CD2CDD2009F429C18091D60181608093DA
:102D4000D601C12C22C1651308C0341306C0D110AE
:102D500004C08091D601D701CCC04D875E87DF8645
:102D6000702F198B088B6D2D89890E94F51488238B
:102D7000E9F1DD20D9F12091D601822F82958F7063
:102D800090E0029774F08091D1019091D2019887E0
:102D90008F8319861B870A872C87CE0107960E948E
:102DA000A91186E0F701A1EDB1E001900D928A959D
:102DB000E1F70E949A150E948C15CC24C394E5C0BB
:102DC000702F198B088B60E089890E94321A292F95
:102DD00022952F7030E0223031050CF0CAC09F7070
:102DE00009F0C4C0805E883008F4CFC0C7010E94DB
:102DF000A911E3CF0817190708F456C0F801E81B1A
:102E0000F90BCF018C32914008F456C0C12C702FC1
:102E1000198B088B6D2D89890E944C15E1EDF1E02D
:102E200086E0DF011D928A95E9F70E948C15ADC0FE
:102E3000651314C0341312C0D11010C08091D60194
:102E4000F7018583C7010E94A91186E0E1EDF1E059
:102E5000DF011D928A95E9F7CB2C97C04D875E87DD
:102E6000DF86702F198B088B6D2D89890E94F514D0
:102E7000882309F4BBCFDD2009F4B8CF2091D60117
:102E8000822F82958F7090E002970CF48ACF809108
:102E9000D1019091D2019A8389831B821D830C8377
:102EA0002E83CE0101967BCF80959095800F911F48
:102EB0008C32914008F0AACFCD2CDD2009F496CFBA
:102EC00065132EC034132CC02091D60120FD1FC0E5
:102ED000822F82958F70D9F0D70115962C93159774
:102EE0008F3049F08F5F982F9295907F822F8F704F
:102EF000892B15968C93C7010E94A91186E0F701D2
:102F0000A1EDB1E001900D928A95E1F78ECF86E0B8
:102F1000F701A1EDB1E001900D928A95E1F735C07E
:102F20004D875E87DF86702F198B088B6D2D898901
:102F30000E94F514811135CF8091D6018160809374
:102F4000D601C7010E94A91120C0DD2009F44ECF8F
:102F50004D875E87DF86702F198B088B6D2D8989D1
:102F60000E94F514882309F441CF1BCF81113ACF79
:102F70000CC0243031050CF039CF9F7009F432CFEA
:102F8000F7019581907F09F02DCF8C2D61960FB6BA
:102F9000F894DEBF0FBECDBFDF91CF911F910F918F
:102FA000FF90EF90DF90CF90BF9008951F93CF9345
:102FB000DF93CDB7DEB72C970FB6F894DEBF0FBE08
:102FC000CDBF4F83588769877A878B879C87CE01CF
:102FD00007960E94F515882369F08F8198852A85C8
:102FE0003B85232BF1F19F3F09F063C08F3F09F030
:102FF00060C037C086E0FE013796DE011196019071
:103000000D928A95E1F76F817885EA85FB85309787
:1030100041F17F3F11F46F3F21F12091A00130E099
:10302000C90101968770992740919F0150E084174C
:10303000950709F447C069837A83FD83EC8396E0A2
:10304000929FD001939FB00D1124AF55BE4FFE014A
:10305000319601900D929A95E1F78093A0010E941C
:103060006B1516E080919F019091A0018917C1F125
:10307000189FC00111248F559E4F0E94F51588237B
:1030800079F1E0919F011E9FF0011124EF55FE4F51
:103090004081518162817381848195810E945B1599
:1030A00080919F0190E001968770992780939F01FE
:1030B000D9CF4F81588569857A858B859C850E94FB
:1030C0005B15CFCF0E94F1141092A00110929F01C6
:1030D000E1EDF1E086E0DF011D928A95E9F7C1CFCD
:1030E0002C960FB6F894DEBF0FBECDBFDF91CF9107
:1030F0001F910895DF92EF92FF920F931F93CF934A
:10310000DF93FC01892B09F48AC0E12CF12CDD242A
:10311000D394EF0121968491853709F461C058F466
:10312000843708F04EC0843008F06AC08130D1F096
:10313000823071F174C0883709F45DC050F486376D
:1031400009F455C0873709F06AC08E2D0E94661BAE
:1031500054C09CE7980F903708F061C08F770E94A9
:103160006F1150C08F010E5F1F4FFE01849190E2DE
:10317000980F983050F48770FD2D01C0FF0F8A958D
:10318000EAF78F2F0E946C1B14C00E94041113C019
:103190008F010E5F1F4FFE01C49180E28C0F8830BB
:1031A00060F4C7708D2D01C0880FCA95EAF70E94A0
:1031B000721B0E949D1BE80125C08C2F0E946F117D
:1031C000FACF9F012E5F3F4FFE01C491CC2369F0DF
:1031D0008FE99FE00197F1F700C00000C150F6CFE2
:1031E0009F012E5F3F4FFE01F490E9010BC00E944A
:1031F000561BE82E07C00E94691B0E949D1B02C03F
:103200000E9404118F2D882341F0EFE9FFE03197F0
:10321000F1F700C000008150F6CFFE017ACFDF91B8
:10322000CF911F910F91FF90EF90DF9008956093E1
:103230005702709358028093590290935A020C944B
:103240001E1C089560935B0270935C0280935D0284
:1032500090935E020C941D1C0F931F9300915B02D0
:1032600010915C0220915D0230915E02602B712B07
:10327000822B932B60935B0270935C0280935D02C0
:1032800090935E021F910F910C941D1C0F931F933E
:1032900000915B0210915C0220915D0230915E0210
:1032A000602371238223932360935B0270935C02FB
:1032B00080935D0290935E021F910F910C941D1CF0
:1032C0000F931F9300915B0210915C0220915D02AD
:1032D00030915E02602771278227932760935B02FB
:1032E00070935C0280935D0290935E021F910F9138
:1032F0000C941D1C60E070E0CB010C9417190F9327
:103300001F9341E050E060E070E08A019B0104C03F
:10331000000F111F221F331F8A95D2F7C901B80170
:103320001F910F910C9417190F931F9341E050E0D8
:1033300060E070E004C0440F551F661F771F8A9538
:10334000D2F78091570290915802A0915902B09102
:103350005A028A019B01082B192B2A2B3B2BC901EE
:10336000B8011F910F910C9417190F931F9341E00F
:1033700050E060E070E004C0440F551F661F771FE7
:103380008A95D2F740955095609570958091570237
:1033900090915802A0915902B0915A028A019B0162
:1033A000082319232A233B23C901B8011F910F9138
:1033B0000C9417190F931F9341E050E060E070E008
:1033C00004C0440F551F661F771F8A95D2F780915E
:1033D000570290915802A0915902B0915A028A0165
:1033E0009B01082719272A273B27C901B8011F91EC
:1033F0000F910C9417190F931F930091570210917E
:1034000058022091590230915A02602B712B822B65
:10341000932B1F910F910C9417190F931F930091E9
:103420005702109158022091590230915A0260239C
:103430007123822393231F910F910C9417190F93DB
:103440001F93009157021091580220915902309118
:103450005A0260277127822793271F910F910C949E
:10346000171908958F929F92AF92BF92DF92EF92B9
:10347000FF920F931F93CF93DF9300D000D01F9242
:10348000CDB7DEB76B837C838D838A018C819D8170
:10349000892B21F01F3F29F44F3F19F480E090E081
:1034A0004CC08B818823C9F180905B0290905C02B4
:1034B000A0905D02B0905E028091570290915802F8
:1034C000A0915902B0915A02882A992AAA2ABB2AA5
:1034D0008FE1E82EF12CD501C4010E2C04C0B69565
:1034E000A795979587950A94D2F780FF07C0DE2CA1
:1034F000B8018E2D0E94571D019729F481E0E81A2A
:10350000F10848F7D12C88E0189FF0011124E00F52
:10351000F11DE952FE4FD08209C088E0189FF001EA
:103520001124E00FF11DE952FE4FD08009831A8368
:1035300069817A818D2D0E94571D0F900F900F90F9
:103540000F900F90DF91CF911F910F91FF90EF900F
:10355000DF90BF90AF909F908F90089590910A0157
:10356000992321F090910B01911109C020910C0138
:1035700030910D01F90132969FEF40E030C0982F55
:103580009695969596959F31A0F4E0910C01F09157
:103590000D01E90FF11D877021E030E0A90102C0A3
:1035A000440F551F8A95E2F7CA019181892B8183C7
:1035B00008959091840290FF23C01F928F938DEE07
:1035C00093E09F938F930E941E060F900F900F9091
:1035D0000F9008959F3F39F04F5F4E3141F0519168
:1035E0005813F8CF0DC05111F7CF942FF5CF9F3F4F
:1035F00039F0F901E90FF11D97FDFA9582830895DD
:10360000089590910A01992321F090910B01911155
:1036100009C020910C0130910D01F9013296205E14
:103620003F4F30C0982F9695969596959F31A8F468
:10363000E0910C01F0910D01E90FF11D877021E07F
:1036400030E0A90102C0440F551F8A95E2F7CA0174
:10365000809591818923818308959091840290FFC0
:1036600016C01F928F938FEC93E09F938F930E94CD
:103670001E060F900F900F900F9008953196E2174D
:10368000F30729F090819813F9CF1082F7CF0895AE
:1036900081E090E0E0910C01F0910D01E80FF91F3D
:1036A0001082019680329105A9F7089580918302D6
:1036B000089590918302892B8093830208958095C9
:1036C00090918302892380938302089580938302DB
:1036D000089510928302089590918202892B80931D
:1036E00082020895809590918202892380938202BC
:1036F0000895109282020895809361020E94941CA2
:103700009093600280935F0208951092610210927C
:10371000600210925F02089580910C0190910D015A
:10372000FC0131969C01205E3F4F80E09191911108
:103730008F5FE217F307D1F70895E0910C01F09144
:103740000D01809183028083E0910C01F0910D01C5
:10375000908180918202892B8083809161028823ED
:10376000D9F10E94941C20915F023091600282176F
:10377000930748F00E94941C20915F0230916002F0
:10378000821B930B0AC00E94941C20915F0230910F
:10379000600220953095820F931F8C32914070F01B
:1037A0008091840280FF08C08BE094E09F938F9308
:1037B0000E941E060F900F900E94851BE0910C0145
:1037C000F0910D01908180916102892B80830E948C
:1037D0008C1B81110E94851B80910C0190910D0121
:1037E0000C940B0F909339018093380108958295C2
:1037F000982F9C7C392F36953695282F237344E0DB
:10380000249FC0011124932F982B292F2A7A2695C3
:10381000892F8575880F822B08950895CF93DF93A4
:1038200000D000D01F92CDB7DEB70F900F900F9051
:103830000F900F90DF91CF910895089508950C9403
:103840008C1080919902843021F11092850220E43D
:1038500088E190E00FB6F894A895809360000FBEC1
:103860002093600083B7817F846083BF83B78160CA
:1038700083BF7894889583B78E7F83BF0FB6F89403
:10388000A89580916000886180936000109260002C
:103890000FBE0895CF930E9432070E9450060E94E7
:1038A0003307C0E08C2F0E942907811104C0CF5F2D
:1038B000C031C1F701C081E0CF9108950E948E1000
:1038C0000C94F1141F920F920FB60F9211248F9344
:1038D0009F93AF93BF9380918502811113C0809114
:1038E000860290918702A0918802B0918902419648
:1038F000A11DB11D8093860290938702A093880238
:10390000B0938902BF91AF919F918F910F900FBE9D
:103910000F901F90189582E084BD93E095BD9AEFBB
:1039200097BD80936E0008952FB7F894809186021A
:1039300090918702A0918802B09189022FBF0895CB
:103940002FB7F89460918602709187028091880267
:10395000909189022FBF0895CF92DF92EF92FF924C
:103960000F931F932FB7F8944091860250918702CE
:1039700060918802709189022FBF6A017B01EE2459
:10398000FF248C0120E030E0C016D106E206F306E9
:1039900010F4415051099A01281B390BC9011F919C
:1039A0000F91FF90EF90DF90CF900895CF92DF922C
:1039B000EF92FF920F931F932FB7F894C090860257
:1039C000D0908702E0908802F09089022FBF970183
:1039D0008601061B170B280B390BC616D706E806FF
:1039E000F90618F0C901B80106C0C901B801615053
:1039F0007109810991091F910F91FF90EF90DF905C
:103A0000CF9008951F920F920FB60F9211248F93AB
:103A10009F93AF93BF938091860290918702A0916C
:103A20008802B09189020196A11DB11D8093860282
:103A300090938702A0938802B0938902BF91AF91BF
:103A40009F918F910F900FBE0F901F9018950E941D
:103A5000180CF8942FEF87EA91E6215080409040AF
:103A6000E1F700C0000087E090EBDC018093A20248
:103A70009093A302A093A402B093A5029CE088E1D6
:103A80000FB6F894A895809360000FBE90936000E5
:103A9000FFCF28E0929FF0011124E80FF11DE052C2
:103AA000FF4F9491892F8F7092959F700895CF93B7
:103AB000C82FCB010E94491D282F30E080E1989F3C
:103AC000A0011124422B532B4038510519F480E0FA
:103AD00090E015C09770E92FF0E088E0C89FE00DF6
:103AE000F11D112484E0EE0FFF1F8A95E1F7E20F2C
:103AF000F31FEE0FFF1FE050F84985919491CF918D
:103B0000089580E090E00895089580918C0280FFF0
:103B10000BC06091110185E0689FB001112475957B
:103B20006795759567952BC081FF09C0609111015C
:103B300085E0689FB00111247595679520C082FFCC
:103B400007C06091110185E0689FB001112417C082
:103B500090918D029923D1F060911001961788F70A
:103B60002091110185E0289F90011124929FA001CE
:103B7000939F500D112470E0CA010E945D256038AA
:103B8000710540F46115710539F002C065E070E01F
:103B9000862F08958FE7089581E0089580918C0223
:103BA00080FF08C060910F0170E07595679575956D
:103BB000679521C081FF06C060910F0170E0759587
:103BC000679519C082FF04C060910F0170E010C0BA
:103BD00090918D029923C1F060910E019617A0F784
:103BE00080910F01899FC001112470E00E945D2522
:103BF0006038710528F46115710521F0862F08954C
:103C00008FE7089581E0089561E070E0F4CF803F90
:103C100021F40E94851D819504C0813F29F40E94F2
:103C2000851D809390020895823F21F40E94851D96
:103C3000819504C0833F29F40E94851D80938F02E3
:103C40000895893F19F40E94CE1D05C08A3F31F4C2
:103C50000E94CE1D81958093910208958B3F21F49F
:103C60000E94CE1D819504C08C3F29F40E94CE1D78
:103C7000809392020895843F21F480918E028160A6
:103C800017C0853F21F480918E02826011C0863F6B
:103C900021F480918E0284600BC0873F21F48091D3
:103CA0008E02886005C0883F31F480918E02806169
:103CB00080938E0208958D3F21F480918C02816063
:103CC0000BC08E3F21F480918C02826005C08F3F33
:103CD00029F480918C02846080938C020895803F47
:103CE00039F48091900287FF6CC01092900269C0F5
:103CF000813F29F4809190021816BCF362C0909124
:103D00008F02823F29F497FF5CC010928F0259C046
:103D1000833F19F41916CCF354C0893F41F48091C4
:103D2000910218160CF04DC0109291024AC08A3FC1
:103D300029F48091910287FF44C0F6CF8B3F39F47C
:103D40008091920287FF3DC0109292023AC08C3F50
:103D500029F4809192021816BCF333C0843F21F4F9
:103D600080918E028E7F17C0853F21F480918E0254
:103D70008D7F11C0863F21F480918E028B7F0BC016
:103D8000873F21F480918E02877F05C0883F31F400
:103D900080918E028F7E80938E0213C08D3F21F41E
:103DA00080918C028E7F0BC08E3F21F480918C021B
:103DB0008D7F05C08F3F29F480918C028B7F80938B
:103DC0008C0280918F0281110EC08091900281112E
:103DD0000AC080919102811106C0809192028111E6
:103DE00002C010928D0208958091840283FF7EC0EC
:103DF00084E494E00E94850580918E021F928F9347
:103E00008FE394E09F938F930E941E068DE394E0CE
:103E10000E94850580918F02282F082E000C330BFD
:103E20003F938F938AE394E09F938F930E941E06A3
:103E300088E394E00E94850580919002282F082E47
:103E4000000C330B3F938F9385E394E09F938F9304
:103E50000E941E0683E394E00E94850580919102F2
:103E6000282F082E000C330B3F938F9380E394E0B0
:103E70009F938F930E941E068EE294E00E94850518
:103E800080919202282F082E000C330B3F938F93C2
:103E90008BE294E09F938F930E941E0688E294E049
:103EA0000E94850580918D021F928F9385E294E098
:103EB0009F938F930E941E0683E294E00E948505E3
:103EC00080918C021F928F9380E294E09F938F9356
:103ED0000E941E068DE194E00E9485058DB79EB775
:103EE0004C960FB6F8949EBF0FBE8DBF8EE892E041
:103EF0000E94540F0E94941C90938B0280938A021C
:103F000008951F93CF93DF9380918A0290918B0243
:103F10000E94AC1CAC0190918D02992321F020915C
:103F2000120130E006C0209113018AE0289F900121
:103F300011244217530708F485C080918F02C09165
:103F40009002D091910210919202811107C0C1118B
:103F500075C0D11173C0111171C074C09F3F19F0A9
:103F60009F5F90938D02181624F40E94851D809304
:103F70008F0280918F0287FF05C00E94851D819569
:103F800080938F021C1624F40E94851D809390025A
:103F90008091900287FF05C00E94851D81958093C6
:103FA000900260918F02662331F1C0919002CC2380
:103FB00011F1062E000C770B880B990B0E945824E8
:103FC00023E333E343E35FE30E94BC240E94202405
:103FD00060938F026C2FCC0F770B880B990B0E948C
:103FE000582423E333E343E35FE30E94BC240E94AD
:103FF0002024609390021D1624F40E94CE1D80930D
:1040000091028091910287FF05C00E94CE1D81958B
:1040100080939102111624F40E94CE1D8093920287
:104020008091920287FF05C00E94CE1D81958093EA
:104030009202DF91CF911F910C94F41E9F3F09F0E3
:104040008FCF97CFDF91CF911F910895EEE8F2E0E7
:1040500085E0DF011D928A95E9F710928D0210929A
:104060008C02089587E696E00E9485051F9281E004
:104070008F931F9285E08F9389E196E09F938F93B2
:104080000E941E060F900F900F900F900F900F90B0
:1040900008958330E9F128F4813061F0823009F12C
:1040A0000895853009F462C008F449C0863009F4E7
:1040B00074C0089580911301262F30E0280F311D20
:1040C0002F3F310524F4680F6093130103C08FEF75
:1040D00080931301809113011F928F9382E595E0E5
:1040E00072C080911201262F30E0280F311D2F3F22
:1040F000310524F4680F6093120103C08FEF8093A1
:104100001201809112011F928F9380E495E05BC0B1
:1041100080911101262F30E0280F311D2F3F3105EE
:1041200024F4680F6093110103C08FEF8093110195
:10413000809111011F928F938DE295E044C0809190
:104140001001262F30E0280F311D2F3F310524F4B8
:10415000680F6093100103C08FEF8093100180916E
:1041600010011F928F9388E195E02DC080910F017F
:10417000262F30E0280F311D2F3F310524F4680F22
:1041800060930F0103C08FEF80930F0180910F01A7
:104190001F928F938FEF94E016C080910E01262F0F
:1041A00030E0280F311D2F3F310524F4680F609354
:1041B0000E0103C08FEF80930E0180910E011F92BC
:1041C0008F9384EE94E09F938F930E941E060F902E
:1041D0000F900F900F900895833081F128F4813073
:1041E00059F08230D1F00895853009F449C0B8F112
:1041F000863009F456C0089580911301681720F4A1
:10420000861B8093130102C0109213018091130149
:104210001F928F9385ED94E054C08091120168172E
:1042200020F4861B8093120102C01092120180912B
:1042300012011F928F9383EC94E043C0809111018F
:10424000681720F4861B8093110102C0109211019F
:10425000809111011F928F9380EB94E032C0809186
:104260001001681720F4861B8093100102C0109281
:104270001001809110011F928F938BE994E021C06F
:1042800080910F01681720F4861B80930F0102C0F4
:1042900010920F0180910F011F928F9382E894E09A
:1042A00010C080910E01681720F4861B80930E01C8
:1042B00002C010920E0180910E011F928F9387E62B
:1042C00094E09F938F930E941E060F900F900F9083
:1042D0000F900895CF93C82F1F928F938CE697E08D
:1042E0009F938F930E941E0681E090E0A0E0B0E0D3
:1042F000BC01CD0104C0660F771F881F991FCA95A6
:10430000D2F70E9422190F900F900F900F90CF912B
:104310000C94F114CF938732A8F58E3108F02BC19D
:10432000803109F49FC0F8F4873009F464C0A8F420
:10433000863009F024C180918402817F8E7F809332
:10434000840281E797E00E9485058BE59AE00E9450
:10435000850581E0809394024CC08B30F1F18E3062
:1043600009F46CC00CC1863109F4B0C020F481316D
:1043700009F4EDC004C1893109F491C08B3109F40D
:1043800049C0FDC0883349F150F4893209F4F1C0C5
:10439000853309F4EEC0873209F0F1C0EAC08334F6
:1043A00009F4E7C028F48A3308F4E9C08953E4C06B
:1043B000883409F0E4C00E94F1148AE49AE00E9473
:1043C00085052FEF83ED90E3215080409040E1F789
:1043D00000C000000E94271D0CC088E997E05CC067
:1043E00081E39AE00E948505809184028160809338
:1043F0008402C1E0C9C080918402C82FC17080FFCF
:10440000EFCF8DE39AE00E94850580918402817F41
:104410008E7F3DC09091840291FBCC27C0F981E052
:10442000C827892FC0FB81F980938402CC2319F01F
:1044300084E29AE027C086E19AE02EC0909184023F
:1044400092FBCC27C0F981E0C827892FC0FB82F9F5
:1044500080938402CC2319F087E09AE013C087EFA1
:1044600099E01AC09091840293FBCC27C0F981E0B7
:10447000C827892FC0FB83F980938402CC2351F095
:104480008BEE99E00E948505809184028160809383
:1044900084027AC08EED99E00E948505AACF8FEC48
:1044A00099E00E94850582EA99E00E9485058BE6E5
:1044B00099E00E9485058EE399E00E94850584EFCE
:1044C00098E00E94850586EC98E0E6CF88EB98E0BE
:1044D0000E9485050E94FF0E1F928F938EE998E03F
:1044E0009F938F930E941E0680910A011F928F93C3
:1044F00087E898E09F938F930E941E068091870122
:104500001F928F9384E798E09F938F930E941E06DB
:1045100080910B011F928F9381E698E09F938F9378
:104520000E941E060E94A01C9F938F937F936F93FF
:104530008AE498E09F938F930E941E068DB79EB7E2
:1045400046960FB6F8949EBF0FBE8DBF52CF0E9405
:10455000F114C0910B0181E0C827C0930B01CC235B
:1045600029F080E498E00E9485050EC085E398E07C
:1045700093CF80E001C08D510E946A213ACF83E33E
:1045800098E00E948505C0E08C2FCF91089580E0CF
:10459000089580E00895CF93C82F809194028130D0
:1045A00071F020F0823009F44BC042C1E0910C015F
:1045B000F0910D018081823209F03CC107C0E09189
:1045C0000C01F0910D018081823261F48C2F0E94E8
:1045D000C722811104C08C2F0E948A212FC081E044
:1045E00090E02CC08C2F0E94C922811126C0C431BA
:1045F000E1F070F4CB3081F0C031D1F40E94322070
:1046000084E697E00E94850582E08093940215C0BD
:10461000C93259F0C83361F481E797E00E948505FB
:1046200088E697E00E94850508C01092940204C1B4
:1046300082E697E00E948505FFC081E08170FEC0A0
:10464000C43228F5CE3108F0C1C0CB30A1F1D0F48E
:10465000C73009F0D3C08EE18093130182E38093C9
:1046600012018AE08093110184E18093100188E0B7
:1046700080930F0188E280930E0188E096E00E940B
:104680008505BFC0C33149F1C431C1F0B7C0CB34D7
:1046900009F4A9C028F4C93289F0C83361F0AEC06A
:1046A000C13509F49EC0C23509F499C0CE3409F071
:1046B000A5C06AE09EC00E943220A3C080919302F0
:1046C000882319F0109293029CC085E196E00E9425
:1046D000850581E080939402B1C08FEE95E00E9441
:1046E00085058DED95E00E948505809113011F924F
:1046F0008F938AED95E09F938F930E941E0688ED1D
:1047000095E00E94850586EC95E00E9485058091E4
:1047100012011F928F9383EC95E09F938F930E94D9
:104720001E0681EC95E00E94850582EB95E00E94D3
:104730008505809111011F928F938FEA95E09F93D9
:104740008F930E941E068DEA95E00E9485058CE9F4
:1047500095E00E948505809110011F928F9389E951
:1047600095E09F938F930E941E0687E995E00E9433
:10477000850582E895E00E94850580910F011F92D2
:104780008F938FE795E09F938F930E941E068DE78E
:1047900095E00E94850586E695E00E94850580915A
:1047A0000E011F928F9383E695E09F938F930E9453
:1047B0001E0681E695E00E9485058DB79EB7489656
:1047C0000FB6F8949EBF0FBE8DBF1BC0CE51EC2F0D
:1047D000F0E0E25DFE4F80818093930212C061E0C1
:1047E00003C061E006C06AE0809193020E94492004
:1047F00008C0809193020E94EC2003C086E096E0FE
:1048000013C080919302882369F01F928F9380E0F8
:1048100096E09F938F930E941E060F900F900F902B
:104820000F9004C08DEF95E00E94850581E006C0E1
:104830001092940280E002C080E000CFCF910895F2
:104840000E9427246894B1110C94B62408950E9404
:104850009B2488F09F5798F0B92F9927B751B0F053
:10486000E1F0660F771F881F991F1AF0BA95C9F7F4
:1048700014C0B13091F00E94B524B1E008950C94B9
:10488000B524672F782F8827B85F39F0B93FCCF36C
:10489000869577956795B395D9F73EF49095809571
:1048A000709561957F4F8F4F9F4F0895E89409C091
:1048B00097FB3EF490958095709561957F4F8F4F53
:1048C0009F4F9923A9F0F92F96E9BB279395F69569
:1048D000879577956795B795F111F8CFFAF4BB0FE7
:1048E00011F460FF1BC06F5F7F4F8F4F9F4F16C04B
:1048F000882311F096E911C0772321F09EE8872FD5
:10490000762F05C0662371F096E8862F70E060E090
:104910002AF09A95660F771F881FDAF7880F969509
:10492000879597F9089557FD9058440F551F59F0F2
:104930005F3F71F04795880F97FB991F61F09F3F8C
:1049400079F087950895121613061406551FF2CFB5
:104950004695F1DF08C0161617061806991FF1CF05
:1049600086957105610508940895E894BB2766272C
:104970007727CB0197F908950E94CF240C94402506
:104980000E94322538F00E94392520F0952311F03D
:104990000C9429250C942F2511240C94B6240E94E4
:1049A000932470F3959FC1F3950F50E0551F629FBC
:1049B000F001729FBB27F00DB11D639FAA27F00D78
:1049C000B11DAA1F649F6627B00DA11D661F829F9F
:1049D0002227B00DA11D621F739FB00DA11D621F84
:1049E000839FA00D611D221F749F3327A00D611DA1
:1049F000231F849F600D211D822F762F6A2F112483
:104A00009F5750409AF0F1F088234AF0EE0FFF1FB5
:104A1000BB1F661F771F881F91505040A9F79E3F0C
:104A2000510580F00C9429250C94B6245F3FE4F3E3
:104A3000983ED4F3869577956795B795F795E79562
:104A40009F5FC1F7FE2B880F911D9695879597F96B
:104A5000089597F99F6780E870E060E008959FEF00
:104A600080EC089500240A94161617061806090605
:104A7000089500240A9412161306140605060895D4
:104A8000092E0394000C11F4882352F0BB0F40F45C
:104A9000BF2B11F460FF04C06F5F7F4F8F4F9F4F9C
:104AA0000895991B79E004C0991F961708F0961B8A
:104AB000881F7A95C9F78095089597FB072E16F4FD
:104AC000009407D077FD09D00E94772507FC05D018
:104AD0003EF4909581959F4F0895709561957F4F15
:104AE0000895EE0FFF1F0590F491E02D0994AA1B85
:104AF000BB1B51E107C0AA1FBB1FA617B70710F0C9
:104B0000A61BB70B881F991F5A95A9F780959095FA
:0A4B1000BC01CD010895F894FFCF19
:104B1A003B072C080908D507A107010162022808EA
:104B2A00140A321E404D3622393703EA02B4029281
:104B3A00025902CC01E501FE011702370200010207
:084B4A00030405060708090039
:1068000088000000000000000400050006000700EA
:10681000080009000A000B000C000D000E000F001C
:1068200010001100120013001400150016001700CC
:10683000180019001A001B001C001D001E001F007C
:10684000200021002200230024002500260027002C
:10685000280035002A002B002C002D002E002F00D0
:1068600030000000320033003400290036003700C9
:106870003800E00000000000000000000000000000
:106880000000000000000000000000000000000008
:1068900000000000000000000000000000004F00A9
:1068A00050005100520000000000000000000000F5
:1068B00000000000000000000000000000000000D8
:1068C00000000000000000000000000000000000C8
:1068D00000000000000000000000000000000000B8
:1068E0000000000000000000890087008A008B0083
:1068F000F1A1E100E200E300F1A1E500E600000003
:106900000100000000000000EA4401000100E24430
:106910000100010001005500460054004A004B00F0
:10692000560057004700480001000100E9440100FB
:106930000100010001000100010001003A003B00DC
:106940003C003D003E003F0040004100420043004B
:10695000580001004C00390001004400450052007D
:1069600001000000010050004F0081404D004E002A
:1069700051000100000000000000000000000000C5
:106980000000000000000000000000000000000007
:1069900000000000000000000000000000004D00AA
:1069A0004A004E004B000000000000000000000004
:1069B00000000000000000000000000000000000D7
:1069C00000000000000000000000000000000000C7
:1069D00000000000000000000000000000000000B7
:1069E000000000000000000049000100010001005B
:1069F0000100010001000100010001000100000090
:00000001FF
